:1000000019C0C2C2EEC11895189518951895189583
:100010001895189518951895189518951895189578
:100020001895189518951895189518951895189568
:10003000189518958FEF8DBFC0EEE8ED4E2E82E03B
:100040008EBFD2E0F2E05F2EEEEFF1E0A0E0B1E093
:1000500088278D933197E9F784B7082E877F84BF6F
:100060008FE18093600087E0809360004FD5662425
:100070008AEB80936600809169008C7F8260809318
:10008000690080916900837F84608093690080E0CB
:100090008093800082E08093810052985398579A11
:1000A000569820983D983C984B9A5A9A5F9A189A7D
:1000B0004E9A359A349A8FE690E0AEE2B1E08D9395
:1000C0009C9388E891E0A3E4B1E08D939C9384E64F
:1000D00090E0A0E2B1E08D939C9300E010E020E07E
:1000E00030E0AAE4B1E00D931D932D933C93ADD283
:1000F000809100018F7B80930001E1E0F0E0AAE4B1
:10010000B1E094E0D6D641E050E060E070E0AAE4CF
:10011000B1E00D911D912D913C9146D609F412C08C
:1001200001E010E020E030E0AAE4B1E00D931D937F
:100130002D933C93E1E0F0E0AAE4B1E094E07BE7AA
:10014000A7D65CD2E7E0F0E0AEE2B1E092E0B1D653
:10015000E9E0F0E0A3E4B1E092E0ABD6EBE0F0E060
:10016000A2E0B1E094E0A5D6EFE0F0E0AEE0B1E0CF
:1001700094E09FD6EBE0F0E0A6E0B1E094E099D601
:10018000EFE0F0E0A2E1B1E094E093D6809181004D
:10019000887F8093810080E090E090938500809339
:1001A0008400789480916F00816080936F00E89A5A
:1001B000E99AA1D48CE0F2D488E0809301015AD36B
:1001C0000027A9E2B0E08C9183FB0EF401E041E04E
:1001D000041709F001C0F4CF81E080930101AEE083
:1001E000B1E04D915D916D917C91AAE1B1E00D91ED
:1001F0001D912D913C91D8D581E009F080E08F933D
:10020000A4E8B0E00D911C9100325EE4150780E097
:1002100010F009F081E09F918923882309F412C02E
:100220000027A0E0B1E08C9186FB0EF401E040E0F5
:10023000041709F007C01ED3E1D18091000180644A
:1002400080930001A0E2B1E04D915C91AEE1B1E09C
:100250000D911C910417150714F009F001C021C07D
:1002600080E090E0AEE1B1E08D939C9303D3002752
:10027000A0E0B1E08C9186FB0EF401E041E00417B0
:1002800009F008C04F9A88E99AE3A0E2B1E08D93A3
:100290009C9306C088E893E1A0E2B1E08D939C9323
:1002A00003C0AEE1B1E0CCD32098A0E0B1E09C91D6
:1002B00095FF04C0189B0EC09F7D9C9318990AC09F
:1002C00089E19F939927EDD49F91189903C090627B
:1002D0009C932FD05698A0E0B1E09C9194FF04C06D
:1002E0004E9B0EC09F7E9C934E990AC089E19F93BE
:1002F0009927D7D49F914E9903C090619C9340D089
:100300003D98A0E0B1E09C9193FF04C0359B0EC0E6
:10031000977F9C9335990AC089E19F939927C1D40F
:100320009F91359903C098609C933AD058CFF89428
:10033000FFCFE1D3A1E0B1E08C918F5F8C930027D8
:10034000A6E2B0E08C9184FB0EF401E041E00417DA
:1003500009F00BC000910101073010F009F001C055
:1003600003C081E0809301010AC0009101010330C4
:1003700010F009F001C003C081E0809301010895ED
:1003800000910101053009F004C0A3E4B1E058D3A5
:1003900006C0063009F003C0AEE2B1E051D30895C3
:1003A00000910101033009F006C04FD127D181E04F
:1003B0008093010115C0053009F004C0A3E4B1E049
:1003C00046D30EC0063009F004C0AEE2B1E03FD320
:1003D00007C0073009F004C011D181E0809301010A
:1003E00008950F921F922F923F924F925F927F92A9
:1003F000AF92BF920F931F932F933F934F935F93AF
:100400006F937F938F939F93AF93BF93CF93DF931C
:10041000EF93FF938FB78F930027A9E2B0E08C9101
:1004200083FB0EF401E040E0041781E009F080E076
:100430008F930027A0E0B1E08C9187FB0EF401E0E0
:1004400040E0041781E009F080E09F918923882330
:1004500009F41BC0809100018068809300015F9ABD
:10046000AEE0B1E00D911D912D913C91AAE1B1E07A
:100470000D931D932D933C9380E090E09093850025
:100480008093840082E0809381000027A9E2B0E09D
:100490008C9183FB0EF401E041E0041781E009F048
:1004A00080E08F930027A0E0B1E08C9187FB0EF4F1
:1004B00001E041E0041781E009F080E09F91892389
:1004C000882309F445C0809100018F778093000153
:1004D0005F98809100018F7B8093000100E010E025
:1004E00020E030E0AAE1B1E00D931D932D933C9301
:1004F00080918100887F80938100A4E8B0E00D9115
:100500001C9100325EE4150708F022C0A4E8B0E0B8
:100510000D911C9148EE53E0C4D2A4E1B0E08D915E
:100520009C919093850080938400A2E0B1E00D91AE
:100530001D912D913C91A4E8B0E04D915C9166270E
:10054000772728D4A2E0B1E00D931D932D933D931E
:100550008F918FBFFF91EF91DF91CF91BF91AF91BD
:100560009F918F917F916F915F914F913F912F91CB
:100570001F910F91BF90AF907F905F904F903F90F1
:100580002F901F900F9018950F921F922F923F92CD
:100590004F925F927F92AF92BF920F931F932F93D0
:1005A0003F934F935F936F937F938F939F93AF93FB
:1005B000BF93CF93DF93EF93FF938FB78F93AEE00B
:1005C000B1E02FD28F918FBFFF91EF91DF91CF914B
:1005D000BF91AF919F918F917F916F915F914F915B
:1005E0003F912F911F910F91BF90AF907F905F909F
:1005F0004F903F902F901F900F901895F8948091F6
:100600008100887F80938100E7E0F0E0AEE2B1E016
:1006100092E07BE73DD4E9E0F0E0A3E4B1E092E0D2
:100620007BE736D4EBE0F0E0A2E0B1E094E07BE7DA
:100630002FD4EFE0F0E0AEE0B1E094E07BE728D427
:10064000789482E080938100089500E010E020E03B
:1006500030E0A2E0B1E00D931D932D933C9300E0B8
:1006600010E020E030E0AEE0B1E00D931D932D935B
:100670003C9300E010E020E030E0A6E0B1E00D9314
:100680001D932D933C9300E010E020E030E0A2E1C8
:10069000B1E00D931D932D933C93089500910101BA
:1006A000013009F019C0A2E0B1E00D911D912D912A
:1006B0003C91AAE0B1E00D931D932D933C93AEE0E5
:1006C000B1E00D911D912D913C91A6E1B1E00D930A
:1006D0001D932D933C9329C0023009F026C0A2E05F
:1006E000B1E00D911D912D913C91A6E0B1E04D91AD
:1006F0005D916D917C9153D3AAE0B1E00D931D9370
:100700002D933D93AEE0B1E00D911D912D913C9163
:10071000A2E1B1E04D915D916D917C9140D3A6E154
:10072000B1E00D931D932D933D93AAE0B1E00D919F
:100730001D912D913C9144E650E060E070E051D273
:10074000AAE2B1E04D935D936D937D93AAE2B1E08F
:100750000D911D912D913C91AEE2B1E04D915D91D5
:1007600057FB1EF46FEF7FEF02C066277727A8D2F2
:10077000AAE2B1E00D931D932D933D93AAE2B1E05F
:100780000D911D912D913C9140E157E260E070E0A8
:1007900028D2A2E2B1E04D935D936D937D93A6E2E2
:1007A000B1E0E2E2F1E016D3A6E1B1E00D911D91D6
:1007B0002D913C91A3E4B1E04D915D9157FB1EF466
:1007C0006FEF7FEF02C0662777277AD2AFE3B1E001
:1007D0000D931D932D933D93AFE3B1E00D911D91CA
:1007E0002D913C91AAE2B1E04D915D916D917C918A
:1007F000F8D1AAE4B1E04D935D936D937D93AEE49F
:10080000B1E0EAE4F1E0E6D2AFE3B1E00D911D9191
:100810002D913C9140EA56E861E070E0E2D1A5E319
:10082000B1E04D935D936D937D93A9E3B1E0E5E372
:10083000F1E0D0D247EE53E060E070E0A2E2B1E038
:100840000D911D912D913C91AFD214F009F001C092
:1008500010C0FBDEA9E3B1E0E0ECFEE054D2AEE470
:10086000B1E0E6ECFEE04FD2A6E2B1E0E6ECFEE05D
:100870004AD2089513DF00910101013009F030C020
:100880003FD1EAECFEE02FD1EEE4F1E0A0ECB2E0E3
:100890001127222703E031E03FD21DD1E6EDFEE033
:1008A00022D127D1EAEDFEE01ED1E9E3F1E0A0EC90
:1008B000B2E01127222705E031E02ED20CD1ECED79
:1008C000FEE011D1E6E2F1E0A0ECB2E01127222730
:1008D00003E031E021D2FFD0E2EEFEE004D19EC081
:1008E000023009F030C00CD1E4EEFEE0FCD0EEE4C2
:1008F000F1E0A0ECB2E01127222703E031E00CD2B6
:10090000EAD0E6EDFEE0EFD0F4D0EAEDFEE0EBD089
:10091000E9E3F1E0A0ECB2E01127222705E031E0A5
:10092000FBD1D9D0ECEDFEE0DED0E6E2F1E0A0ECC8
:10093000B2E01127222703E031E0EED1CCD0E2EE85
:10094000FEE0D1D06BC0033009F009C0D9D0E0EF90
:10095000FEE0C9D0CED0E2E0FFE0C5D05FC00430F9
:1009600009F015C0CDD0E4E1FFE0BDD0A0ECB2E0CD
:10097000EEE0F1E02FD2AFD0BCD0EAE1FFE0B3D09F
:10098000A0ECB2E0E2E0F1E025D2A5D047C005300E
:1009900009F015C0A5E4B1E0E3E4F1E020D2B0D065
:1009A000E0E2FFE0A0D0A5D0E5E4F1E0A0ECB2E009
:1009B00010E1222704E03327AFD18DD02FC00630BD
:1009C00009F015C0A0E3B1E0EEE2F1E008D298D062
:1009D000E2E3FFE088D08DD0E0E3F1E0A0ECB2E00C
:1009E00010E1222704E0332797D175D017C00730D4
:1009F00009F009C085D0E4E4FFE075D07AD0E6E5DF
:100A0000FFE071D00BC0083009F008C079D0E8E6EB
:100A1000FFE069D06ED0EAE7FFE065D00895F89472
:100A2000FFCF0D911D912D913C9181E0080F8827FA
:100A3000181F281F381F3C932E931E930E93089562
:100A4000ED91FC91EF5FFF4FFC93EE930895ED91D4
:100A5000FC91E150F040FC93EE93089500FC10D01F
:100A6000089503D01ED001F8F9CF0024E89457FF71
:100A700002C009D0689400F80BD010F80124089542
:100A800002D009D00895509540954F5F5F4F08956B
:100A9000E89417FF0895009510950F5F1F4F689415
:100AA0000895352F242FE894452B11F46894089568
:100AB000512F402F0027112780E1440F551F001FA1
:100AC000111F021B130B416018F4020F131F4E7FFE
:100AD0008A9599F70895A0ECB2E08D91882311F0E2
:100AE00057D0FBCF089514D1802D11F051D0FBCFFA
:100AF000089580EC53C081E051D005D080E84EC00D
:100B000080E84CD0089583E09927CBC08AEF90E02D
:100B1000C8D0219A229A239A249A259A559A5D98A8
:100B200085E090E0BED02D9829982A982B9A2C9A8F
:100B30002D9AEF93FF93E4ECF0E0A7D0FF91EF91B3
:100B40002D98ACD02D9AEF93FF93E4ECF0E09DD07C
:100B5000FF91EF912D98A2D02D9AEF93FF93E4ECA3
:100B6000F0E093D0FF91EF912D9898D02C982D9A8A
:100B7000EF93FF93E4ECF0E088D0FF91EF912D9894
:100B80008DD088E20BD08EE009D086E007D00895A2
:100B90005D9A829505D004D081D008955D98F9CFF3
:100BA000859510F42C9A01C02C98859510F42B9AF9
:100BB00001C02B98859510F42A9A01C02A98859532
:100BC00010F4299A01C029982D9AEF93FF93E4EC31
:100BD000F0E05BD0FF91EF912D98089500FC05D0D7
:100BE000089530D005D001F8F9CF37D03FD008951F
:100BF000842F952FA62FB72FE894452B462B472BF4
:100C000011F468940895402F512F622F732F0027FD
:100C1000112722273327F0E2440F551F661F771F45
:100C2000001F111F221F331F081B190B2A0B3B0B20
:100C3000416028F4080F191F2A1F3B1F4E7FFA95A9
:100C400059F708950024E89477FF02C006D068940D
:100C500000F809D010F80124089512D04F5F5F4FBB
:100C60006F4F7F4F0895E89437FF089500951095D2
:100C7000209530950F5F1F4F2F4F3F4F6894089579
:100C8000409550956095709508953197F1F70895C6
:100C9000689462F80895E89462F8089581E090E01D
:100CA00000C0EF93FF93EE27E82BE92B31F0E0ED46
:100CB000F7E03197F1F70197D1F7FF91EF910895A0
:100CC0000F921F922F92C801D901489F80014A9F1D
:100CD00090014B9F202C499F100D211D321D5A9FC2
:100CE000202C589F100D211D321D599F200D311DA4
:100CF000689F200D311D699F300D789F300D2F901A
:100D00001F900F90089504D00D920020E1F70895F0
:100D1000C8953196002008952E2E3F2E9927819157
:100D20008D3209F093958823D1F79A95E22DF32D12
:100D3000112361F0091718F011F0101B01C0191BE5
:100D400028F021F080E28D931A95E9F780818D32A9
:100D500019F48D93319604C0222311F08BE28D9308
:100D6000091738F031F0091B21F080E38D930A95C3
:100D7000E9F781918D938823E1F7332351F0EA2F2E
:100D8000FB2F319633958E9182933A95E1F78EE25F
:100D90008C930895040F151F261F371F0895041BF9
:100DA000150B260B370B0895041715072607370771
:100DB0000895000F111F221F331F089500951095ED
:100DC000209530950F5F1F4F2F4F3F4F0895019192
:100DD00010810EC001911191219130810BC00191C0
:100DE000108117FF05C03FEF2FEF04C000811127CE
:100DF0002227332737FF03C0E1DF8DE28D93CF93A6
:100E0000DF93CF92DF92EF92AA24BB24CC24DD247F
:100E1000EE2440E2CAE0DD2755E093E38881890FA4
:100E200087FD9F7083FD907F891B89935A95A9F751
:100E3000C0DFAA1CBB1CCC1CDD1CEE1C4A9551F764
:100E4000E894EFE0FF2782910ED0EB30E0F71EF040
:100E500068948A2D0CD088278D93EF90DF90CF90E7
:100E6000DF91CF910895982F829501D0892F8F70AF
:100E7000805D26F0803309F4089568948D93089579
:100E8000F999FECFE1BD3196089591E001C092E05D
:100E90007B3751F47FB7F894F3DF8D9180BDFA9AD8
:100EA000F99A9A95C9F77FBF7727089591E001C015
:100EB00092E0E6DFF89A80B58D939A95D1F7089580
:100EC0002D2D2D2D2D002D2D2D00BADEB3B9B2C83C
:100ED000DDCBDF2000004B6D000052004B6D204643
:100EE00000004C00BADDB6B2C8DDCBDF2020000028
:100EF0002D4441544120434C454152204F4B3F2DFE
:100F00000000446F776E4B4559203D20434C4541CE
:100F1000522000005350443D0000494E4A3D00001D
:100F20005345542053706565642050554C53202020
:100F3000000053455420496E6A6563742050756CF7
:100F4000732000002D4441544120575249544520FC
:100F50004F4B3F2D0000446F776E4B4559203D208D
:100F600057726974652000002D2DC8DDCBDF20B9D4
:100F7000B2BFB8D4DBB32D2D000050524F475241C1
:0C0F80004D20566572312E31334A0000BE
:00000001FF
